:020000020000FC
:100000000FC047C147C17EC17FC16CC17EC17EC1E7
:0E0010007EC179C165C165C17BC17BC17BC169
:10002000F89411E00EE51EBF0DBF00E811E006BD1B
:1000300016BD08E008BB07E107BBF0E0E0E600E022
:100040000193E036E9F7F130D9F700E00BBF00E0AB
:1000500009BF08E005BB00E60ABF06E408BF00E0F0
:1000600005BF02E000BD00E00ABD05E003BF00E0FF
:1000700002BF00E009BD00E008BD0CE60CBD00E0D9
:100080000EBD00E00BBD0FEF0DBD00E007BD05EE9E
:1000900000BF00EA07B900E003B907EE06B900E2C5
:1000A00004BB00E808B9A89504B7077F04BF01B5F1
:1000B000006101BD0EE401BD00E20BBF02E009BF1B
:1000C0000CE8202E0EE6302E0DE7402E0CE8502EC8
:1000D0000EEB602E0CE3702E04E1802E0FE0902ECC
:1000E00070E080E190E083E080D10F3F59F0302E46
:1000F00084E07BD1402E85E078D1502E86E075D10A
:10010000602E08C00EE6302E0DE7402E0CE8502E73
:100110000EEB602E7894A89507E107BB90FFFBCF0C
:100120009E7F04E1802E91FD04C07A9409F49260D0
:100130004AC004B700FF06C00E7F04BF022D043B77
:1001400008F042C004B105B1093B10F00FE0902E59
:10015000251408F414C0022D0519033008F42CC02E
:1001600016B31A7F146018BB10E01BBD162D1519AD
:1001700014501DBD035092FF00E00EBD24C0052D9C
:100180000219033008F418C016B31A7F116018BBA7
:1001900010E01EBD152D131914501DBD035010E0A5
:1001A000252D241930E0C9D0252D231930E0E0D0C9
:1001B00092FF00E00BBD07C0946016B31A7F18BB16
:1001C00000E00EBD0BBDA7CF07EE00BF04E60DBDDE
:1001D00008E2E8D0022D0093660001E09CD002E323
:1001E000E1D0022D003808F02BC00093630075EABF
:1001F00001E091D002E3D6D0022D0093650001E02A
:100200008AD002E3CFD0022D10916300011710F4C1
:10021000012F06C010916500011710F0012F00C0DA
:100220000093640001E077D002E3BCD0022D10916E
:100230006600011B08F40195053008F001C012C0EA
:1002400070E001E068D002E0ADD001E064D002E0EF
:10025000A9D001E060D002E0A5D001E05CD00AE0C6
:10026000A1D0FDCF0091630083E0B0D00091640085
:1002700084E0ACD00091650085E0A8D000916600D4
:1002800086E0A4D070E080E10AE045D00AE08AD0A0
:10029000FDCF1895FFB666B363FD20C0F0E0E0E047
:1002A0000000000066B363FD03C03196B9F0F8CFDB
:1002B00060E0E1FD61E0F695E795F695E795E60FDC
:1002C000E21559F028F06FEF261639F0239405C097
:1002D00062E3261611F02A9400C09160FFBE1895C3
:1002E00018951895FFB69A9419F49B7F6FE0962E97
:1002F0008A9431F466B36A7F68BB60E06EBD6BBD03
:10030000FFBE189518951895189518951895189575
:100310001895189518951F9316B31A7F146018BB7B
:1003200010E01BBD15E01EBD3DD016B31A7F18BBF3
:1003300010E01BBD1EBD1F9108954F935F936F93F7
:10034000551B441B61E110F4400F511F5795479511
:10035000379527956A95B9F75F934F933F932F93FE
:100360000F911F912F913F916F915F914F91089540
:100370004F935F936F934427552760E1000F111F40
:10038000441F551F4217530718F00395421B530B88
:100390006A95A1F75F934F932F913F916F915F9172
:1003A0004F9108951F932F931CE920E00000000057
:1003B0000000000000000000A8952A95B9F71A95E2
:1003C000A1F70A9589F72F911F9108951F93E1993D
:1003D000FECF10E01CBB10E01FBB8EBB0DBB753AFF
:1003E00011F4E29AE19A1F9108951F93E199FECFCB
:0E03F00010E01FBB8EBBE09A0DB31F91089565
:00000001FF
